:040000008A116A2FC8
:100E0000FE00FE1F082F83137E18831700080800BA
:100E10000408FE0007308A007E0882070034FC3494
:100E2000123412341234FC347E088A007F088200A7
:100E300014278A118000840A04087D0603190034EF
:100E4000FF0A0319FE0A182F64008001840A0406B1
:080E5000031900340406252FEC
:100EAA00632FF930F4006400F40B582F5C2F6400B0
:100EBA00FF30F5070318F60AFF30F60776087504BF
:100ECA00031D682F692F562F0800FA01FB01FC0148
:100EDA00FD0183134030840050308A1124278A117F
:100EEA004030FD000730FE008330FF0020308400D0
:100EFA008A1118278A1183018A11A32F30343134B9
:100F0A00323433343434353436343734383439348B
:100F1A00413442344334443445344634EE34ED34B7
:100F2A00EB34E734DE34DD34DB34D734BE34BD345D
:100F3A00BB34B7347E347D347B347734981307302E
:100F4A00831603139C0003100030031801309D0020
:100F5A0003100030031801309B001830850003107D
:100F6A0000300318013086000310003003180130E6
:100F7A008312031385000310003003180130860022
:100F8A008312031385140330F700F70BCA2F831259
:100F9A00031385100030F8000030F90083120313A0
:100FAA0005150330F700F70BD82F83120313051129
:100FBA007808013E8A1109278A1186000230F50055
:100FCA000030F6008A1155278A110130F8070318F4
:100FDA00F90A0030F9077908803AF7008030770279
:100FEA00031DF92F05307802031CFC2FFD2FD32F88
:060FFA00C52F8A1100283A
:00000001FF
